:1000000012C0189518951895189518951895189563
:1000100078C11BC1189518951895189518951895BD
:100020001895189518958FE58DBFC8E3E4EF4E2E0F
:1000300084E08EBFD4E0F3E05F2EEEEFF3E0A0E6C5
:10004000B0E088278D933197E9F784B7082E877F32
:1000500084BF8FE181BD87E081BD662483E083BFDB
:1000600080E08FBD83E08EBD8EB5887F8EBD8CED28
:100070009BE090934D0080934C008FEF87BB8FEFF8
:1000800081BB80E084BB8FEF85BB80E08093600004
:1000900080E08093610080E08093620080E0809344
:1000A0006300A198A4E6B0E09C9197FF04C0999BDF
:1000B0000EC09F779C9399990AC089E19F939927D5
:1000C000B4D19F91999903C090689C9348D0A0980F
:1000D000A4E6B0E09C9196FF04C0989B0EC09F7B65
:1000E0009C9398990AC089E19F9399279ED19F91EB
:1000F000989903C090649C9355D0A298A4E6B0E070
:100100009C9195FF04C09A9B0EC09F7D9C939A99E9
:100110000AC089E19F93992788D19F919A9903C03A
:1001200090629C9362D0009163000C3309F004C08C
:1001300080E08093630027D1009160000A3009F0CD
:1001400003C080E080936000009161000A3009F0F4
:1001500003C080E080936100A4CFF894FFCF0091AA
:100160006200003009F00AC089B7816089BF7894C5
:10017000A0E6B0E08C918F5F8C93C19A00916200F1
:10018000013009F00EC080E08093620089B78B7F58
:1001900089BF8EB5887F8EBDA0E6B0E08C918F5F61
:1001A0008C93089500916200003009F00AC089B76D
:1001B000816089BF7894A1E6B0E08C918F5F8C93C9
:1001C000C29A00916200013009F00EC080E0809375
:1001D000620089B78B7F89BF8EB5887F8EBDA1E60F
:1001E000B0E08C918F5F8C93089500916200003095
:1001F00009F010C0F89480E088BB88EC90E015D13D
:10020000789489B7846089BF83E08EBD81E0809354
:10021000620015C080E08093620089B78B7F89BF40
:100220008EB5887F8EBD80E08093600080E08093F3
:10023000610080E08093620080E080936300089515
:10024000B7067357C6D5F507F7D70F921F922F92AF
:100250003F924F925F927F92AF92BF920F931F9304
:100260002F933F934F935F936F937F938F939F93BE
:10027000AF93BF93CF93DF93EF93FF938FB78F939A
:1002800082EB809352000027A8E3B0E08C9181FBC1
:100290000EF401E041E0041709F00CC0E0E4F2E0E4
:1002A000A0E6B0E08C919927A2E3B0E0DDD0C19840
:1002B000C29A0BC0E0E4F2E0A1E6B0E08C9199278D
:1002C000A2E3B0E0D1D0C298C19A8F918FBFFF91C5
:1002D000EF91DF91CF91BF91AF919F918F917F91DE
:1002E0006F915F914F913F912F911F910F91BF900F
:1002F000AF907F905F904F903F902F901F900F9006
:1003000018950F921F922F923F924F925F927F9279
:10031000AF92BF920F931F932F933F934F935F938F
:100320006F937F938F939F93AF93BF93CF93DF93FD
:10033000EF93FF938FB78F938CED9BE090934D00DD
:1003400080934C00A3E6B0E08C918F5F8C938F91EB
:100350008FBFFF91EF91DF91CF91BF91AF919F91AF
:100360008F917F916F915F914F913F912F911F914D
:100370000F91BF90AF907F905F904F903F902F90E4
:100380001F900F90189500916100003081E009F0F6
:1003900080E08F9300916000013081E009F080E0FF
:1003A0009F918923882309F40EC089B78B7F89BF69
:1003B0008EB5887F8EBD80E080936200C09A80E415
:1003C00096E033D0C09800916000003010F009F042
:1003D00001C006C0809160008150809360001BC006
:1003E00000916000003081E009F080E08F9300917F
:1003F0006100003080E010F009F081E09F918923D6
:10040000882309F408C080916100815080936100C5
:1004100089E08093600008953197F1F7089568941A
:1004200062F80895E89462F80895EF93FF93EE2739
:10043000E82BE92B31F0E8EEF3E03197F1F7019783
:10044000D1F7FF91EF910895C89531960020089556
:1004500091E005C092E003C094E001C098E0F4DFB1
:0E0460000D929A95E1F70895E80FF91FF1CF7C
:00000001FF
